:100000003FC2000059C2000057C2000055C20000A4
:1000100053C2000051C200004FC200004DC2000098
:100020004BC2000049C2000047C200000C94610AA4
:1000300043C2000041C200003FC200003DC20000B8
:100040003BC2000039C2000037C2000035C20000C8
:1000500033C2000031C200002FC200004CC60000B5
:100060002BC2000029C2000027C2000025C20000E8
:1000700023C2000021C200001FC200001DC20000F8
:100080001BC2000019C2000017C2000015C2000008
:1000900013C2000011C2000005010905A1011500ED
:1000A0002501350045017501951005091901291033
:1000B000810205012507463B017504950165140978
:1000C00039814265009501810126FF0046FF000944
:1000D000300931093209357508950481020600FF9F
:1000E0000920950181020A212695089102C012017A
:1000F0000002000000400D0F92000001010200010B
:100100000902290001010080FA090400000203002D
:1001100000000921110100012256000705020340D9
:10012000000507058103400005040309041C03487A
:10013000004F0052004900200043004F002E002CC9
:10014000004C00540044002E000000240350004FD7
:10015000004B004B0045004E00200043004F004E76
:1001600000540052004F004C004C0045005200006B
:10017000001032000A020010C80012020010320003
:100180000A020010320010320012020010140001A6
:100190000500100200030200100500030200100514
:1001A000000302001005000A0500103C000A0200CE
:1001B000101E000A0200101E001014000A05001094
:1001C00014000805001014001205001014000A05A0
:1001D000001014000A05001014000A050010140095
:1001E0000A05001014000A05001014000A0500108A
:1001F00014000A05001014000A05001014000A0576
:10020000001014000A05001014000B050010460031
:100210000A02001032000B02001032000B02001024
:1002200032000B02001032000B02001032000B02F1
:10023000001032000A02001032000A020010AF0063
:100240001205001014000202001008000102000252
:1002500002000A0200102D00010200140200010237
:100260000014020001020014020001020014020046
:100270000102001402000102001402000102001435
:1002800002000102001002000A0200100F00010229
:10029000001402000119001402000102000A020009
:1002A000100A000102001402001002000A020010ED
:1002B0000A000302001602000002000302001602F8
:1002C000000302001002000A0200101400120500D0
:1002D0001023001205001023000B02001028000A52
:1002E00002001064001005000A02001014000A0247
:1002F000001014000A02001014000B020010140079
:100300000B02001014000B02001014000B0200106E
:1003100014000B02001014000B02001014000B025A
:10032000001014000B02001014000B020010140047
:100330000B02001014000B02001014000B0200103E
:1003400014000B02001014000B02001014000B022A
:10035000001014000B02001014000B020010140017
:100360000B0200101400120500101400020200100D
:1003700008000102000202000A0200102D00010222
:100380000014020001020014020001020014020025
:100390000102001402000102001402000102001414
:1003A00002000102001402000102001002000A0211
:1003B00000100F00010200140200011900140200D5
:1003C0000102000A0200100A0001020014020010DB
:1003D00002000A0200100A000302001602000002D6
:1003E000000302001602000302001002000A0200CD
:1003F0001014001205001023001205001023001035
:100400000A000202001502000202001502000202A8
:1004100000000200030200160200030200160200A0
:100420000302001002000A02001004000A02001079
:10043000040002020015020002020015020002027E
:100440000001E6000302001602000302001602008B
:100450000302001002000A02001004000A02001049
:1004600004000B02001014000002001004000A0532
:10047000001004006364696E6F70737578585B00D8
:1004800011241FBECFEFD2E0DEBFCDBF11E0A0E050
:10049000B1E0E2EBF0E202C005900D92AA3BB10799
:1004A000D9F712E0AAEBB1E001C01D92A432B10766
:1004B000E1F729D50C945710A3CD80E88093D201A1
:1004C0008093D3018093D4018093D50188E08093F9
:1004D000D101089508950895FB018C3009F470C08E
:1004E0008D3058F5853009F479C0863098F4823023
:1004F00009F453C0833038F4882309F471C0813083
:1005000009F097C073C0833009F449C0843009F002
:1005100090C062C0883009F44BC0893038F486300E
:1005200009F463C0873009F084C05CC08A30D1F11F
:10053000208131818B30D0F53FC0843109F476C001
:100540008531A8F48F3009F458C0803130F48D30F3
:10055000D9F18E3009F06DC04CC0823109F451C020
:10056000833108F05DC0813109F063C031C087314B
:1005700009F452C0883138F4853109F448C0863115
:1005800009F057C046C0893109F44FC0893108F4D9
:1005900045C08A3109F04DC045C0138208958FEFE0
:1005A000838308958081918184602EC0226005C07C
:1005B00080819181886028C02160318320830895E3
:1005C00080819181806120C08081918180621CC086
:1005D00080819181806318C0138202C08FEF838372
:1005E000148208958FEF838302C013828FEF848378
:1005F000089580819181926007C08081918191608E
:1006000003C08081918190619183808308951582D8
:1006100008958FEF85830895158202C08FEF85833B
:10062000168208958FEF858302C015828FEF86832F
:10063000089580E8838384838583868388E082832A
:1006400008950F931F93CF93DF93FC018B01EA0171
:100650002091FC013091FD018091010290910202F4
:1006600063E070E00E94C90C2F5F3F4F3093FD01A3
:100670002093FC0121503040281739074CF4DE014B
:10068000E1ECF1E088E001900D928150E1F7A2C029
:100690001092FD011092FC014091FE015091FF016A
:1006A0008091FA019091FB01841795079CF01092BC
:1006B000FB011092FA0180E88B838C838D838E83FB
:1006C00088E08A83A1ECB1E0FE0101900D92815097
:1006D000E1F781C09C012F5F3F4F3093FB012093D6
:1006E000FA018091C9019091CA01A091CB01B0910A
:1006F000CC010097A105B105D9F12131310551F5A2
:100700000197A109B1098093C9019093CA01A093EF
:10071000CB01B093CC010097A105B10539F481E27A
:1007200090E09093FB018093FA012BC02091BD01D2
:100730003091BE012B33310524F581E090E0909398
:10074000FB018093FA012F5F3F4F3093BE0120934E
:10075000BD0117C021323105A1F481E090E09093F2
:10076000FB018093FA011092BE011092BD0109C0F5
:100770002417350734F0415050405093FB0140930B
:10078000FA018091FA019091FB0163E070E00E9410
:10079000C90CE80FF91F87EF91E0BF0143E050E07B
:1007A0000E94DB0C1093FF010093FE018091F80181
:1007B0009091F90190930202809301028091F701D8
:1007C000BE018ADEA1ECB1E0FE0188E001900D924D
:1007D0008150E1F781E0DF91CF911F910F91089552
:1007E0000F931F93CF93DF93FC018B01EA012091BC
:1007F000FC013091FD01809101029091020263E0C1
:1008000070E00E94C90C2F5F3F4F3093FD01209391
:10081000FC0121503040281739074CF4DE01E1EC8F
:10082000F1E088E001900D928150E1F750C0109204
:10083000FD011092FC012091FA013091FB018091A1
:10084000FE019091FF01281739079CF01092FB01DF
:100850001092FA0180E88B838C838D838E8388E0ED
:100860008A83A1ECB1E0FE0101900D928150E1F785
:100870002FC02F5F3F4F3093FB012093FA0121508F
:100880003040C90163E070E00E94C90CE80FF91F15
:1008900087EF91E0BF0143E050E00E94DB0C109332
:1008A000FF010093FE018091F8019091F90190936E
:1008B0000202809301028091F701BE010DDEA1ECDE
:1008C000B1E0FE0188E001900D928150E1F781E0F6
:1008D000DF91CF911F910F910895CF93DF93EC019A
:1008E00098E0FE01892F11928A95E9F780E88B83C1
:1008F0008C838D838E839A838091BB018130C1F07C
:10090000813030F0823009F1833009F0A0C09CC002
:100910001092FB011092FA018FE790E09093FF0193
:100920008093FE018091BF01882369F081E08DC032
:100930006091A8017091A90181E791E0AE0150DFBB
:10094000882309F084C082E080C08091BC0185309A
:1009500009F444C0863070F4823029F1833020F4E9
:10096000813009F074C018C0833051F1843009F02F
:100970006EC02DC0883009F44EC0893030F4863006
:10098000B1F1873009F063C039C0893009F44AC039
:100990008A3009F05CC04FC06091AC017091AD012C
:1009A00089EB91E045C06091B2017091B3018BEC8D
:1009B00091E0AE0115DF8CEA8B8387E08C8347C022
:1009C0006091B4017091B5018DE092E031C0609109
:1009D000B6017091B70185EE92E02AC06091B8012E
:1009E0007091B9018FEF93E0AE012BDE30C06091C2
:1009F000A8017091A90181E791E006C06091AA0168
:100A00007091AB0186E891E0AE01EADE8823F9F44B
:100A10001092BC011CC06091AE017091AF018FEBD0
:100A200091E006C06091B0017091B10185EC91E058
:100A3000AE01D6DE0CC0DE01EFECF1E088E0019003
:100A40000D928150E1F703C084E08093BB01DF91F8
:100A5000CF910895EF92FF920F931F93DF93CF935F
:100A6000CDB7DEB763970FB6F894DEBF0FBECDBF2C
:100A70007C0100D000D000D0EDB7FEB73196ADB705
:100A8000BEB712969C938E93119780E091E093836A
:100A900082838E010C5F1F4F15830483EAD72DB725
:100AA0003EB72A5F3F4F0FB6F8943EBF0FBE2DBF33
:100AB0008F5F9F4F11F488E001C1C80163E071E0CE
:100AC00040E150E081D7009721F41092BC01F5DCA1
:100AD000F7C08C8180538A3008F079C01092D00121
:100AE0001092CF018DB79EB740970FB6F8949EBF76
:100AF0000FBE8DBFEDB7FEB73196ADB7BEB712963C
:100B0000FC92EE92119787E091E093838283CE016D
:100B1000029695838483CE0101969783868380E035
:100B200092E09187808780EC91E0938782878EECBA
:100B300091E0958784878DEC91E09787868799D798
:100B400089818093D1014A815B81642F6170CA01E0
:100B5000969587952DB73EB7205F3F4F0FB6F89417
:100B60003EBF0FBE2DBF282F217080FF08C080918F
:100B700000028093D2018091C0018093D301862F1F
:100B800090E030E082239323892B39F08091CE01CD
:100B90008093D4018091CD0108C0662341F08091FB
:100BA00000028093D4018091C0018093D5015695B5
:100BB0004795569547958091CF019091D001482B4C
:100BC000592B5093D0014093CF018AE077C06091B8
:100BD000660170916701C80140E150E0F5D60097C9
:100BE00011F481E06BC06091680170916901C801E6
:100BF00040E150E0E9D6009711F482E05FC06091D7
:100C00006A0170916B01C80140E150E0DDD60097A8
:100C100011F483E053C060916C0170916D01C801C3
:100C200040E150E0D1D6009711F486E047C06091D2
:100C30006E0170916F01C80140E150E0C5D6009788
:100C400011F487E03BC06091700170917101C8019F
:100C500040E150E0B9D6009711F484E02FC0C801FC
:100C600064E271E044E050E0AFD6009731F585E0F2
:100C70008093BC0100D000D000D0EDB7FEB7319614
:100C8000ADB7BEB71296FC92EE92119789E291E051
:100C90009383828389EC91E095838483EAD61092D2
:100CA000BE011092BD012DB73EB72A5F3F4F0FB670
:100CB000F8943EBF0FBE2DBF03C089E08093BC01F6
:100CC0001092FB011092FA018FE790E09093FF01E0
:100CD0008093FE01109202021092010263960FB6F9
:100CE000F894DEBF0FBECDBFCF91DF911F910F9162
:100CF000FF90EF9008951F920F920FB60F9211245C
:100D00000F931F932F933F934F935F936F937F9313
:100D10008F939F93AF93BF93EF93FF9380911E02A6
:100D200090911F025FD6082F8091C80085FF03C0F5
:100D3000802F90E099D60D3061F407ED11E0C801E5
:100D400089DE1092BA0180E2F80111928A95E9F7E2
:100D50000EC00A3061F08091BA01803240F4E82F71
:100D6000F0E0E952FE4F00838F5F8093BA01FF915C
:100D7000EF91BF91AF919F918F917F916F915F9113
:100D80004F913F912F911F910F910F900FBE0F9098
:100D90001F901895FF920F931F93DF93CF93CDB7BA
:100DA000DEB728970FB6F894DEBF0FBECDBF809197
:100DB00007028430B9F582E08093E9008091E80071
:100DC00082FF14C08091E80085FF0BC08E010F5F89
:100DD0001F4FC80167E070E040E050E0FBD188237E
:100DE000C1F78091E8008B778093E80081E08093E1
:100DF000E9008091E80080FF15C08E010F5F1F4F52
:100E0000C8016BDDF02E012F8F2D902F68E070E070
:100E100040E050E031D28823B9F78091E8008E7726
:100E20008093E80028960FB6F894DEBF0FBECDBFC2
:100E3000CF91DF911F910F91FF9008950F931F9312
:100E4000DF93CF93CDB7DEB728970FB6F894DEBF08
:100E50000FBECDBF80910902813019F0893051F564
:100E600016C080910802813A29F58E010F5F1F4F4D
:100E7000C80133DD8091E800877F8093E800C801D6
:100E800068E070E09FD08091E8008B7711C080917E
:100E90000802813279F48091E800877F8093E8002E
:100EA000CE01019667E070E0F1D08091E8008E7786
:100EB0008093E80028960FB6F894DEBF0FBECDBF32
:100EC000CF91DF911F910F91089582E060EC42E392
:100ED00025D281E061EC42E321C284B7877F84BFE1
:100EE00088E10FB6F89480936000109260000FBE06
:100EF00080E090E020E80FB6F894209361008093A2
:100F000061000FBECFC287E690E09093CD00809342
:100F1000CC0086E08093CA001092C80088E18093DC
:100F2000C900539A5A9A80E090E015D57894809140
:100F3000C90080688093C900C0DACFDF78942ADFC7
:100F4000D7D4FDCFDA019330B1F0943028F491304A
:100F500041F0923079F50AC0913211F1923251F597
:100F600024C0EEEEF0E022E130E028C0E0E0F1E065
:100F700029E230E023C0813049F0813018F082301E
:100F8000C9F40AC0E9E2F1E0849103C0EDE2F1E0C6
:100F90008491282F30E012C0EBE4F1E08491F9CF86
:100FA000E2E1F1E029E030E009C0E8E9F0E026E51F
:100FB00030E004C0E0E0F0E020E030E0ED93FC93AE
:100FC000C90108959C0140910E0250910F024617ED
:100FD000570718F4F90190E03DC06115710511F053
:100FE000AB01F8CF8091E8008E778093E80040E075
:100FF00050E0F0CF80910702882309F441C085308A
:1010000009F440C08091E80083FD3EC08091E80073
:1010100082FD30C08091E80080FF1CC08091F2000A
:10102000282F30E007C081918093F100415050405B
:101030002F5F3F4F4115510519F02034310598F3CA
:1010400090E02034310509F491E08091E8008E773A
:101050008093E8004115510569F6992359F60AC0B5
:1010600080910702882361F0853061F08091E8006B
:1010700083FD0AC08091E80082FFF2CF80E00895EE
:1010800082E0089583E0089581E008959C01611550
:10109000710529F48091E8008B778093E800F901CD
:1010A00020C080910702882361F1853061F1809131
:1010B000E80083FF02C081E008958091E80082FF8C
:1010C000F0CF06C08091F10081936150704021F013
:1010D0008091F2008823B1F78091E8008B778093AC
:1010E000E80061157105E9F606C0809107028823C2
:1010F00041F0853041F08091E80080FFF6CF80E03C
:10110000089582E0089583E008959C0140910E02C5
:1011100050910F024617570718F4F90190E03EC0AE
:101120006115710511F0AB01F8CF8091E8008E7761
:101130008093E80040E050E0F0CF809107028823E0
:1011400009F442C0853009F441C08091E80083FD74
:101150003FC08091E80082FD31C08091E80080FFAF
:101160001DC08091F200282F30E008C08491809348
:10117000F1003196415050402F5F3F4F41155105CE
:1011800019F02034310590F390E02034310509F452
:1011900091E08091E8008E778093E8004115510539
:1011A00061F6992351F60AC080910702882361F005
:1011B000853061F08091E80083FD0AC08091E800ED
:1011C00082FFF2CF80E0089582E0089583E00895E1
:1011D00081E00895BF92CF92DF92EF92FF920F933A
:1011E0001F93CF93DF93182F092F7B016A01EFD054
:1011F000B82E8823B1F5812F902F9C01E901C114ED
:10120000D10439F0F60180819181E81AF90AC80FFA
:10121000D91F00E010E022C08091E80085FD16C0D3
:101220008091E8008B778093E80062D3C114D104E9
:1012300049F0F60180819181800F911F9183808315
:1012400085E010C0C4D0882349F00CC08091F10023
:1012500089930894E108F1080F5F1F4FE114F1042E
:10126000D9F68B2DDF91CF911F910F91FF90EF90C9
:10127000DF90CF90BF900895BF92CF92DF92EF9210
:10128000FF920F931F93CF93DF93182F092F7B01AA
:101290006A019DD0B82E8823B1F5812F902F9C0133
:1012A000E901C114D10439F0F60180819181E81A75
:1012B000F90AC80FD91F00E010E022C08091E800B1
:1012C00085FD16C08091E8008E778093E80010D3EA
:1012D000C114D10449F0F60180819181800F911FE2
:1012E0009183808385E010C072D0882349F00CC0C0
:1012F00089918093F1000894E108F1080F5F1F4F76
:10130000E114F104D9F68B2DDF91CF911F910F914C
:10131000FF90EF90DF90CF90BF900895382F282F47
:101320002EC0822F8F708093E900231721F4762F2F
:10133000942F50E006C07091EC009091ED00509118
:10134000F00091FF1BC08091EB008E7F8093EB003B
:101350008091ED008D7F8093ED008091EB008160A6
:101360008093EB007093EC009093ED005093F000AD
:101370008091EE0087FD02C080E008952F5F253048
:1013800080F23F703093E90081E008958091080277
:1013900088239CF404C0809107028823B9F08091CF
:1013A000E80082FFF8CF8091E8008B778093E80017
:1013B000089580910702882349F08091E80080FF1A
:1013C000F8CF8091E8008E778093E80008954091EF
:1013D000E4005091E50024E68091EC0080FF24C0F9
:1013E0008091E80080FD1EC080910702882311F4DF
:1013F00082E00895853011F483E008958091EB0038
:1014000085FF02C081E008958091E4009091E5009D
:101410008417950709F3222311F484E008952150DD
:10142000AC01DACF80E008958091E80082FFDCCF44
:10143000F9CF41D043D08091D8008F778093D800E6
:101440008091D80080688093D8008091D8008F7DEB
:101450008093D80084E089BD86E089BD09B400FE90
:10146000FDCF109207021092030210920502109213
:10147000040280E060E042E351DF8091E1008E7F72
:101480008093E1008091E20081608093E20080918E
:10149000E20088608093E2008091E0008E7F80937C
:1014A000E0000895E3E6F0E080818E7F808381E0B4
:1014B00080930602BECF1092E20008951092E100E0
:1014C00008951F920F920FB60F9211242F933F93FE
:1014D0004F935F936F937F938F939F93AF93BF933C
:1014E000EF93FF938091E10082FF0AC08091E200B8
:1014F00082FF06C08091E1008B7F8093E100F7D1ED
:101500008091E10080FF18C08091E20080FF14C04C
:101510008091E2008E7F8093E2008091E200806102
:101520008093E2008091D80080628093D80019BC3B
:10153000109207020E946B028091E10084FF30C08C
:101540008091E20084FF2CC084E089BD86E089BDE3
:1015500009B400FEFDCF8091D8008F7D8093D80024
:101560008091E1008F7E8093E1008091E2008F7E88
:101570008093E2008091E20081608093E20080919C
:101580000302882311F084E007C08091E30087FD07
:1015900002C081E001C083E0809307020E946A02DA
:1015A0008091E10083FF22C08091E20083FF1EC092
:1015B0008091E100877F8093E10082E080930702C1
:1015C000109203028091E1008E7F8093E100809170
:1015D000E2008E7F8093E2008091E2008061809340
:1015E000E20080E060E042E399DE81D1FF91EF917B
:1015F000BF91AF919F918F917F916F915F914F912B
:101600003F912F910F900FBE0F901F9018951F9331
:10161000DF93CF93CDB7DEB7AC970FB6F894DEBFAC
:101620000FBECDBFE8E0F2E08091F100819322E0AF
:10163000E031F207C9F702DC8091E80083FF3FC187
:101640008091080230910902353009F48DC036309E
:1016500040F43130E1F1313070F0333009F02FC116
:1016600036C0383009F4FDC0393009F40CC13630C9
:1016700009F025C19CC0803821F0823809F01FC1D3
:1016800008C090910402809105028823B1F0926015
:1016900014C080910C028F70853008F010C18093C7
:1016A000E9008091EB0090E025E0969587952A95DA
:1016B000E1F7982F91701092E9008091E800877F00
:1016C0008093E8009093F1001092F100D5C0882338
:1016D00019F0823009F0F3C090E08F71907000979C
:1016E00021F0029709F0EBC00CC080910A02813012
:1016F00009F0E5C010920502333081F580930502B0
:101700002DC080910A02882349F520910C022F7088
:10171000822F8150843008F0D2C02093E90080915C
:10172000EB0080FF1BC0333021F48091EB0080621E
:1017300013C08091EB0080618093EB0081E090E02A
:1017400002C0880F991F2A95E2F78093EA00109251
:10175000EA008091EB0088608093EB001092E90032
:101760008091E800877F8BC0882309F0A8C0109182
:101770000A021F778091E3008078812B8093E30039
:101780008091E800877F8093E80000DE8091E80088
:1017900080FFFCCF8091E30080688093E3001123F9
:1017A00011F482E001C083E08093070288C0805872
:1017B000823008F084C080910A0290910B0223E0ED
:1017C0008C3D920709F033C083E08C838AE28B83DF
:1017D0007FB7F894DE0115966EE040E050E011E22C
:1017E000E62FF0E010935700849140FF03C08295EC
:1017F0008F706F5F8F70282F30E08A3018F0C9012A
:10180000C79602C0C901C0968D939D934F5F5F4FED
:101810004431510529F77FBF8091E800877F80938D
:10182000E800CE0103966AE270E0CCDB14C0609160
:101830000C0270910D02AE014F5F5F4F83DBBC0164
:10184000009709F43CC08091E800877F8093E8000E
:1018500089819A815ADC8091E8008B778093E80037
:101860002EC0803861F58091E800877F8093E80082
:10187000809103028093F1008091E8008E7780933D
:10188000E80084DD1CC08823D1F490910A029230D4
:10189000B0F48091E800877F8093E8009093030282
:1018A00075DD80910302882331F48091E30087FD88
:1018B00002C081E001C084E08093070206DB8091D2
:1018C000E80083FF0AC08091E800877F8093E800EA
:1018D0008091EB0080628093EB00AC960FB6F89499
:1018E000DEBF0FBECDBFCF91DF911F910895089548
:1018F0001F9380910702882371F01091E900809175
:10190000EC001092E9008091E80083FF01C07FDEC7
:101910001F701093E9001F910895982F8091C800BF
:1019200085FFFCCF9093CE0080E090E008958091F9
:10193000C80087FD03C02EEF3FEF0BC08091C800A9
:1019400087FD03C02FEF3FEF04C08091CE00282F0A
:1019500030E0C9010895FC01009759F480E192E05C
:1019600090931F0280931E02909321028093200285
:10197000FC018EE0DF011D928A95E9F783E0838305
:101980008DE89CE09187808787E99CE09387828738
:1019900008955527002480FF02C0060E571F660FCA
:1019A000771F6115710521F096958795009799F736
:1019B000952F802D0895FB01DC0102C005900D924A
:1019C00041505040D8F70895FB01DC014150504090
:1019D00030F08D910190801919F40020B9F7881B1F
:1019E000990B0895CF93DF93EC014B8140FF1AC010
:1019F00046FF0AC04F7B4B838E819F8101969F8358
:101A00008E838A81282F2BC042FF13C0E881F98181
:101A10008081282F332727FD30952115310529F4A2
:101A200040624B832FEF3FEF1BC03196F983E88371
:101A300011C0EA85FB85CE0109959C0197FF0AC07C
:101A40009B812F5F3F4F11F080E201C080E1892B25
:101A50008B83E8CF8E819F8101969F838E8330E0B8
:101A6000C901DF91CF910895609120027091210208
:101A70009EC2AEE0B0E0EEE3FDE0F2C285E08C8312
:101A80008B899C899A8389839E01295E3F4FCE0171
:101A900001966D897E89A90176D12E96E2E0FCC27D
:101AA000FC0120FD08C023FD05C022FF02C0738396
:101AB0006283518340830895EF92FF920F931F93A7
:101AC00044FF02C033E011C046FF02C034E00DC045
:101AD000DB01FC01AA0FBB1FEE1FFF1F1094D1F703
:101AE0006A0F7B1F8E1F9F1F31E0660F771F881FB5
:101AF000991F3150D1F77B018C01E20EF11C011DC1
:101B0000111DA8019701B701CA011F910F91FF9004
:101B1000EF9008950F931F93CF93DF938C01C8012B
:101B200061DFEC0197FD06C02FD2892BC1F7CE01F2
:101B3000B80169D2CE01DF91CF911F910F91089525
:101B4000A0E0B0E0E5EAFDE083C2EC01C62E5A0158
:101B5000122F48DFAC018B3219F08D3249F4106836
:101B6000CA9409F466C0CE013DDFAC0197FD61C0A7
:101B70006DEFD62ED1228D2D8073F1F44033E1F438
:101B8000CA9409F442C0CE012DDFAC0197FD3DC0DF
:101B900082E0D82A483711F0483551F480E4D82A39
:101BA000CA9499F1CE011EDFAC0199232CF42DC00B
:101BB000D6FC02C080E1D82AEE24FF248701242F1E
:101BC0002053283080F0D4FC09C02A3060F0D6FEC3
:101BD00005C02F7D822F8151863020F0CA01BE01C1
:101BE00012D210C02750C801B7014D2D65DF7B010F
:101BF0008C0182E0D82ACA9459F0CE01F3DEAC0100
:101C000097FFDDCFD1FC04C014C0EE24FF24870170
:101C1000D7FE08C010950095F094E094E11CF11CEB
:101C2000011D111DC501B801A7012D2D39DF81E06E
:101C300001C080E0CDB7DEB7EAE026C2A0E2B0E0A6
:101C4000E3E2FEE001C26C01A62E8A017901FE01E9
:101C5000319680E2DF011D928A95E9F770E030E06D
:101C600060E040E050E04F01A1E0B0E0F601838188
:101C7000F70183FD259183FF21917F01222309F440
:101C80007CC02E3519F44115510569F1872F90E07C
:101C90008417950744F42D3551F12D3221F4332367
:101CA00029F431E021C0332309F4622F322F832F2E
:101CB000869586958695F401E80FF11D832F877030
:101CC0003D0102C0660C771C8A95E2F72081262927
:101CD0002083361711F430E007C0361710F43F5F49
:101CE000E6CF3150E4CF71E04F5F5F4FBFCF33237A
:101CF00019F08E8180628E83772359F0FE01319630
:101D00009E012F5D3F4F808180958193E217F307FD
:101D1000D1F7BB24B3944E010894811C911CC601D9
:101D200061DEAC0197FD21C0869586958695F4010C
:101D3000E80FF11D808190E09A012770307002C099
:101D4000959587952A95E2F780FD04C0CA01B601F2
:101D50005AD10BC00115110519F0D8014D938D0111
:101D6000AA94BB24AA20D9F602C0BB2031F40115E5
:101D7000110529F0F801108202C0EE24FF24C701EA
:101D8000A096EEE07DC1A0E0B0E0E8ECFEE05CC132
:101D90005C016B013A01FC01178216828824DCC0C9
:101DA000812F90E0F1D0892B19F0C501B3DED4C0AA
:101DB000153249F4F601F3FC6591F3FE61916F0170
:101DC000653259F415E2C5010DDE97FDD1C0181733
:101DD00009F4C2C0B50117D1D0C06A3219F0162F6C
:101DE00000E006C0F3FC1591F3FE11916F0101E0D4
:101DF00099240EC00260692D70E080E090E040E21E
:101E00005BDE962EF601F3FC1591F3FE11916F0146
:101E1000212F20532A3070F301FD03C099249A9496
:101E200003C0992009F4A9C0183621F01C3699F492
:101E3000F6010BC0F601F3FC6591F3FE6191683683
:101E400019F06F01162F07C008600460F3FC1591AC
:101E5000F3FE11916F01112309F48FC084E794E020
:101E6000612F70E099D0892B09F487C0802F00FF83
:101E700003C0EE24FF2407C0F301E080F18022E0DC
:101E800030E0620E731E1E3649F4F501468157811B
:101E900060E070E0C701202F03DE5EC0133689F4D6
:101EA00081FD02C099249394C5019CDD97FD60C01B
:101EB000E114F10419F0F70181937F019A94A1F7DD
:101EC00049C01B3551F4C501692DA7019601B6DE45
:101ED0006C01009709F03EC038C0C5011BDE97FDBC
:101EE00047C01F3641F1103728F4143611F1193666
:101EF00021F524C0133719F01537F9F41AC0C501BC
:101F000071DDEC0197FD0FC03FD0892B21F0CE0190
:101F1000B50179D008C0E114F10419F0F701C193BB
:101F20007F019A9461F7E114F104A1F0F7011082A6
:101F300011C0006203C0006101C00064C501692DC9
:101F4000A701202FFDDD882329F4F501838180730B
:101F500079F413C000FF8394F501F380F601F3FCDC
:101F60001591F3FE11916F01112309F019CF05C0EE
:101F7000882019F42FEF3FEF02C0282D30E0C9016F
:101F8000CDB7DEB7EEE07CC0911157C0803219F0BA
:101F900089508550D0F70895FC010590061621F070
:101FA0000020D9F7C00108953197CF0108950F930C
:101FB0001F93CF93DF938C01EB018B8181FF1BC0BB
:101FC00082FF0DC02E813F818C819D8128173907AA
:101FD00064F4E881F9810193F983E88306C0E88518
:101FE000F985802F0995892B31F48E819F81019687
:101FF0009F838E8302C00FEF1FEFC801DF91CF9147
:102000001F910F9108959C01FB01838180FF11C0F6
:1020100086FD0FC09FEF2F3F390759F02283806460
:102020008F7D83838681978101979783868330E0B4
:1020300002C02FEF3FEFC90108959927882708951F
:102040002F923F924F925F926F927F928F929F92C8
:10205000AF92BF92CF92DF92EF92FF920F931F93B6
:10206000CF93DF93CDB7DEB7CA1BDB0B0FB6F89467
:10207000DEBF0FBECDBF09942A88398848885F84A7
:102080006E847D848C849B84AA84B984C884DF8018
:10209000EE80FD800C811B81AA81B981CE0FD11DFC
:1020A0000FB6F894DEBF0FBECDBFED010895F894D2
:0220B000FFCF60
:1020B200257300656E64002568782025686878209D
:1020C2002568687820256868782025686878202542
:1020D2006868780059656172005965617220256CE3
:1020E20075006D6173685F61006175746F5F6C6527
:1020F2006167756500696E665F77617474007379F4
:102102006E6300756E73796E63007069636B7570D0
:102112006265727279003201390145014E01530143
:102122005A01000000000000000000000000000052
:10213200000000000000000000000000000000009D
:10214200000000000000000000000000000000008D
:10215200000000000000030007001100020002005E
:0A2162000200160048005E0027008E
:00000001FF
